:030000000219FDE5
:03000B000200A848
:03002B0002018847
:03005B0002033964
:030073000203265F
:1000800002030406080C10182030406080040608A3
:100090000C10182030406080A0C00003070F1F051F
:1000A000050D050305030302C2AF306308C2638573
:1000B000798AD2AF32C0D0C0E0206221E525601637
:1000C000E473E525F4C3334009758A00D263F579FA
:1000D00001D4F58AD262D0E0D0D0D2AF32C3E526C7
:1000E000334009758A00D263F57901EEF58AC26260
:1000F000E526F4603030682620720DD0E0D0D0C202
:1001000095C294C293D2AF32C295C294C293206F6B
:100110000D20650A7414D5E0FDE57BF45290D0E023
:10012000D0D0D2AF32758A00D263757900C28DD239
:1001300062211E01C2306805206502D29501C230DD
:100140006805206502D29401C2306805206502D29C
:100150009301C2D29230680A2065077410D5E0FD81
:10016000D29501C2D29130680A2065077410D5E09B
:10017000FDD29401C2D290D29230680A20650774F1
:1001800010D5E0FDD29301C2C2AFC2AD53E6EFC0BD
:10019000D0C0E0D2D3D2AFE57A6009E577600575CB
:1001A000770041D3757701C2CEE52A600720744FEE
:1001B000152A21FF7800790020742EE580307E0119
:1001C000F430E70278FF53DACF207E0343DA2030A1
:1001D0007E0343DA10C2D8C271E580307E01F4306C
:1001E000E70279FFC3E89970CB306103752A1820C4
:1001F0007403752A18885CD270E86003755F00206C
:10020000740DE52B6004152B410F43DA01C2D82091
:1002100070024182A85C206102C270207431C3E880
:1002200094F0400374F0F8E8C4540F28F87984B7C8
:100230000302414FC313C3138721200802C31320B5
:100240000A06C3C898F8414F28F8500374FFF8C352
:10025000E895655003E565F88822E52D540660228F
:10026000206B1FE536C333C333F8E564C313C313F0
:10027000F9C3952240028922E82522F52250037510
:1002800022FF852224A824C3E52495614002A861A9
:100290008825E566700241C6C3E8AA669A5003E85D
:1002A000FAE4F9EAC333FBE568F45B29400D2567FE
:1002B000F8E56760021567400B41C60AC3E5679A17
:1002C0005002056778FF8826C26FC3E52694F84080
:1002D00002D26F20CF0AD0E0D0D043E610D2AD32A8
:1002E000C2CF053AE57A6009E57860057578006166
:1002F0001C7578017801E52A6005307402152AC35F
:10030000E55C94014005755F00611C7560007569CE
:1003100000E55F2401F55F5003755FFFD0E0D0D0AA
:1003200043E610D2AD32C2AF53E67F7592FA7593B1
:10033000FFC260759104D2AF32C2AF53E6EFC2ADD7
:10034000C0D0C0E0C0F0D2D3D2AFA8FBA9FCE57A00
:100350006007C3E913F9E813F8C2D830710261AB42
:1003600053DACF207E0343DA10307E0343DA20D203
:1003700071E580307E01F420E702618288278928B8
:10038000A1D853DACF207E0343DA20307E0343DA4C
:1003900010C2D8C271307402A1C47800E580307EEA
:1003A00001F430E702A1C4885CA1AC53DACF207E0F
:1003B0000343DA20307E0343DA10C27120610281E8
:1003C0008453DACF207E0343DA10307E0343DA20F1
:1003D000C2D8D27188578958C3E89555F8E995561F
:1003E000F97B007E087A00C3E8948CE994005005FC
:1003F000755B008176882178A2E6A8216055C3E864
:1004000094C8E994005008E4D2E4FB7A0A8151C30D
:10041000E89468E994015008E4D2E3FB7A0F815133
:10042000C3E894D0E994025008E4D2E2FB7A1E813A
:1004300051C3E894A0E994055008E4D2E1FB7A3C6A
:100440008151C3E89498E994085008E4D2E0FB7A1B
:10045000787E00C3E89559FCE9955AFD30E70AEC2F
:10046000F42401FCEDF43400FD755B00C3EC9AED5F
:0D0470009E5003755B018859895A855755C8
:10047D008558567802A1ACC3E89527F8E99528F977
:10048D00307C02A190307B02A190307A02A18920AC
:10049D00750281A7E9FDE8FC81C6E9C313F9E813EC
:1004AD00F8307902A189E9C313F9E813F83078021D
:1004BD00A189E9C313FDE813FC20612CC3EC941C46
:1004CD00ED9402400281DDED701EC3EC94C850180E
:1004DD000529E52970021529C3E529940A5002A1C1
:1004ED00C4755C00D270A1C4E52960021529788815
:1004FD00E6F97400207F087896B90302789EE62409
:10050D00FAFEE43400FFC3EC9EFCED9FFD9208B9AA
:10051D000310A2085007207609D276A12F3076025B
:10052D00C276A2085016B9030DECF42401FCEDF4CB
:10053D003400FD02054978007900A190B90315EC4E
:10054D0033FCED33FDC3EC940AFCED9400FD500437
:10055D007C007D00C3EC94FFED9400400678FF799C
:10056D0000A190EC8572F0A4C5F0A2F733F87900E4
:10057D0040030205AC78FF79000205ACE9C313F91D
:10058D00E813F8307C0EE9600278FFC3E81338F801
:10059D00E43400F9C3E894FFE99400400278FF8841
:1005AD005CD270206102A1C4741FF4552F4BF52F3E
:1005BD00C274EB7002D274752A18307403752A0A4E
:1005CD00306102A1D820740353DAFE207403752B19
:1005DD0006D0F0D0E0D0D0D2AD43E6103279010292
:1005ED0006087903020608790A020608791E020632
:1005FD0008796402060879C80206087817E4D5E080
:10060D00FDD8FAD9F6227A147B7802062F7A107B60
:10061D008C02062F7A0D7BB402062F7A0B7BC80253
:10062D00062FE573D5E001227902E4D291D5E0FDE4
:10063D00D294D5E0FDC294D5E0FDC291D5E0FDE99F
:10064D0020E002D29530E002D293E573D5E0FDE9CA
:10065D0020E002C29530E002C2937496D5E0FDD938
:10066D00C9EAF8D5E0FDD8FBDBB8D29122C37C00F6
:10067D007D0075F00005F0EA33FAEB33FB50F6EB35
:10068D0013FBEA13FAC3E9FFE8FEE89AF8E99BF9D0
:10069D005004EFF9EEF8B3EC33FCED33FDD5F0DF9C
:1006AD00EDF9ECF822E889F08A20D2D4F8A9F07B94
:1006BD000030F70B7BFFF42401F8E9F43400F9E87E
:1006CD008520F0A4ADF0F8E98520F0A4AFF0FEEDA3
:1006DD002EF974003FFA7C04C3EA13FAE913F9E822
:1006ED0013F8DCF48BF030F70AE8F42401F8E9F4A0
:1006FD003400F9E889F0C2D4F8A9F02222C3E5410B
:10070D0013F9E54013F8C3E54498F8E54599F95018
:10071D000CC3E89480E994FF4016020741C3E894A6
:10072D007FE994005003020741787F790002074169
:10073D00788079FF8849894A22E5492546F8E54AB6
:10074D003547F9854A20E4300701F43548FA30E79A
:10075D0009C3EA94F0401502077FC3EA940F5003D2
:10076D0002077F78FF79FF7A0F02077F7800790003
:10077D007AF0C3E5249561500AC374019524500B9A
:10078D0002079DE54A20E70E02079DE54A30E70680
:10079D00884689478A482278A5E6FAC3E54933F8A1
:1007AD00E54A33F9D1B2E930E70BC3E89480E99417
:1007BD00FF4013E1D7C3E8947FE994005002E1D7DD
:1007CD00787F7900E1D7788079FFE820E715C3E5D8
:1007DD002398F84009C3E8940140030207FE78010D
:1007ED000207FEE8F424012523F840030207FE78F2
:1007FD00FF884B2278A6E6FAA847A9481206B2E967
:10080D0030E70CC3E89401E994FF4016020833C3A6
:10081D00E894FFE99400500302083378FF79000251
:10082D000833780179FFE920E715C3E54B98F840C7
:10083D0009C3E89401400302085A780102085AE8F6
:10084D00F42401254BF8400302085A78FF8824222E
:10085D0078FF20692879A1E76023E541601F74FFC7
:0F086D008541F0848539F0306A0375F005A4F8F1
:10087C00C5F0600278FFC3E895645002A8648863F1
:10088C0022C3E54094C8E5419400E563500314018C
:10089C009E046002F563220208A62275E890227875
:1008AC0083E6FF30EDF9A8BDA9BE0570C3E57094D1
:1008BC00084052757000E9FA79A0E76044EA7007C5
:1008CC00E571601B0208DFC3E895716010E571509B
:1008DC0006600C140208EB0460F90208EBE571F5F4
:1008EC0071C39472401B7561C0C39404401375614D
:1008FC0080C39404400B756140C39404400375613C
:10090C000075BB0622E561F460020561E570B40771
:10091C000375BB1022743279A787F0A4C5F0A2F737
:10092C0033F8C3E895614002A861882288248825A1
:10093C0088268864227540007541F022C2AF75C8C4
:10094C0020A8CCA9CDAA3A30CF010A75C824D2AFC1
:10095C00C3EA13FAE913F9E813F8AB3BAC3C883B58
:10096C00893CC3E89BF8E99C20690A547FF93066FE
:10097C0002416721C1AD3D8A3DF9EA9D547FFA6081
:10098C000678FF79FF21A6AE3EAF3F8B3E8C3FA889
:10099C003BA93CC3E89EF8E99FF9C3E54113FBE58D
:1009AC004013FAE82AF540E93BF54150067540FF43
:1009BC007541FF410EAA40AB41AC40AD417E047F76
:1009CC0002C3EB9404400D1E1FC3EB94084005209A
:1009DC006A021E1FC3ED13FDEC13FCDEF7C3EA9C89
:1009EC00FAEB9DFBEF6009C3E913F9E813F8DFF7A5
:1009FC00EA28FAEB39FB8A408B4150067BFF8B408F
:100A0C008B41C3EB94025002D2663069047F0341E0
:100A1C00397892E6FFC3E537948240110FC3E5376E
:100A2C0094A040010FC3EF940640027F057E02E5BF
:100A3C0041C4540FF9E541C454F0F8E540C4540FD7
:100A4C0028F8C3E89EFAE99400FB4009C3EA940233
:100A5C00EB940050047A02E4FB41B3AA40AB41EBA7
:100A6C00C4FEEAC4540F4EFCC3EA9CFAEB9400FBA0
:100A7C00C3E813C313F8EA28FAEB3400FB8A408B63
:100A8C0041C3EB94024002C2667802EBC4FE7B00C9
:100A9C00EAC4540F4EFAC3EA98FA4005C3940250C4
:100AAC00027A027892E6FF30600241B3855192855A
:100ABC005293D26043E680C3E49AF8E49BF9C3E80E
:100ACC0033F8E933F93066026146E8FAE9FBD3E919
:100ADC0013FDE813FC88518952C3EF94036038EF7F
:100AEC0020E00DE82CF8E93DF9ECFAEDFB020B0FD8
:100AFC00E828F8E939F9C3E82402F8E93400F97A6E
:100B0C00FE7BFFC3EF9403400E8A538B54884D89B0
:100B1C004E8C4F8D50617A885389548A4D8B4E8CF4
:100B2C004F8D503069127553F07554FF754FF07539
:100B3C0050FF7551F07552FF617AE8FAD3E813FC57
:100B4C008851C3EF94036020EF20E007E82CF8EC09
:100B5C00FA6166E8282402F87AFEC3EF9403400891
:100B6C008A53884D8C4F617A88538A4D8C4FE56837
:100B7C00C3335002646BF5683060026184753402D3
:100B8C00D26043E680E52D5406602DA840A941C3F0
:100B9C00E913F9E813F8306904E92440F9C2AF53BA
:100BAC00E67F759100C3E498F594E499F5957591F9
:100BBC0004D26043E680D2AF22D264754300752024
:100BCC0000306C03752040020BE4D2647543007551
:100BDC002040306C0375200078017901206620E5F7
:100BEC002D54066002C2647914E541C313700104EC
:100BFC00F8C3941440027814306904781B791BC331
:100C0C00E833F8C3E933F9206010E543600C306930
:100C1C0003D53404D26D819A718C0543E59B544005
:100C2C00B52002818430690908C3E8994001188114
:100C3C001320640A08C3E899400261E48113C2647A
:100C4C00C2AF53E67F7591003066127594007595AE
:100C5C00F0759104D26043E680D2AF61E4E5417E49
:0F0C6C00FFC3334009C3334005C3334001FEC308
:100C7B00E49E759400F595815DC3E53394015002B4
:100C8B0061E430640261E4D80281988113C26DC2C1
:100C9B00AF53E67F759100855394855495759104F8
:100CAB00854D92854E93D26043E680D2AFE52D54AD
:100CBB00066008206A020533020CD6306D0D206CDD
:100CCB000A206407158115810215B3227800306460
:100CDB00027801E53775F007A4F9E5F028F5F0E99E
:100CEB00A2F013A2F113A2F213F537C394785003B9
:100CFB00753778C3E53795384008D265C295C294ED
:100D0B00C293306002A10D854F92855093D2604300
:100D1B00E68022207D16C2AF754202D291C292307C
:100D2B006202D293D2AF759F11020F16C2AF7542FA
:100D3B0002D291C290306202D295D2AF759F11024E
:100D4B000F16307245207D22C2AF754203900164AD
:100D5B00757B02C293D290D292306204D294A16D71
:100D6B00C291D2AF759F01020F16C2AF75420390AD
:100D7B000164757B02C295D292306204D294A18D2C
:100D8B00C291D2AF759F21020F16207D17C2AF758E
:100D9B00420390013FC293306202D294D2AF759F4F
:100DAB0001020F16C2AF75420390013FC29530622C
:100DBB0002D294D2AF759F21020F16207D16C2AFBF
:100DCB00754204D292C290306202D294D2AF759F18
:100DDB0021020F16C2AF754204D290D292C292304A
:100DEB006202D294D2AF759F01020F16307243206C
:100DFB007D20C2AF754205900153757B04C294D21E
:100E0B0091306204D295C115C292D2AF759F110277
:100E1B000F16C2AF754205900175757B01C294D256
:100E2B0091306204D293C135C290D2AF759F11023B
:100E3B000F16207D17C2AF754205900135C2943055
:100E4B006202D295D2AF759F11020F16C2AF7542D7
:100E5B0005900149C2943062EBD293D2AF759F11CA
:100E6B00020F16207D18C2AF754206D290D292C2E5
:100E7B0091306202D295D2AF759F01020F16C2AFAD
:100E8B00754206D292C291306202D293D2AF759F55
:100E9B0021020F16307246207D20C2AF75420190A1
:100EAB000175757B01C295D292306204D293C1BD9C
:100EBB00C290D2AF759F21020F16C2AF754201903F
:100ECB000153757B04C293D290D292306205D295B6
:100EDB00020EE0C292D2AF759F01020F16207D1752
:100EEB00C2AF754201900149C295306202D293D2D2
:100EFB00AF759F21020F16C2AF754201900135C22B
:100F0B0093306202D295D2AF759F01C265229001D8
:100F1B0033757B00C295C294C293D292D291D29078
:100F2B00C26222788076FF0876FF0876FF0876FF8C
:100F3B0008760308760408760A0876030876010813
:100F4B007601788C76010876FF0876FF0876FF0825
:100F5B0076FF0876FF0876030876FF0876FF08769B
:100F6B00FF0876250876D00876FA0876FA08760414
:100F7B000876FF08760108760008767A0876FF086F
:100F8B007601087601087600087603087600227849
:100F9B0087E6FFC272BF0302D2727888E6C394035E
:100FAB006008C27DE630E102D27DC27E7889E630F0
:100FBB00E102D27EC3EF94026008758E01D27302F8
:100FCB000FD2758E00C273227880E6149000809346
:100FDB0078A5F67881E6149000809378A6F678864B
:100FEB00E61490008D9378A7F67886E6F539C394CE
:100FFB00025003753902789CE67538FFB40203750D
:10100B0038A0B4030375388278A3E61490009A9342
:10101B00F566120F1922227896E6FA7897E6FB7896
:10102B0088E6B40305C3EB940EFB307F047A007B98
:10103B00FFC3EB9AFCC3948250027C82757200054D
:10104B0072EC8572F0A4C3E5F0947D40F222D27F5E
:10105B0011221205F91205F97A007B007C1012059A
:0F106B00EFE55C2AFA74003BFBDCF37C04C3EB7B
:10107A0013FBEA13FADCF7FEC27F112222757C0009
:10108A00757D00E5EF20E6037520000520903FFFFF
:10109A00E520146006901FFF146000930460037536
:1010AA00EF1653D9BF7581C043FF801205EA75EF69
:1010BA000643B203E5B3240220E70DF521E5E32058
:1010CA00E0068521B343E301120F197580FF75A469
:1010DA000075F19075D47F75908775A5BF75F2BFBD
:1010EA0075D50075A60175E241120F19E4F8F6D814
:1010FA00FD756801120F2E12160D789886737530D9
:10110A0001C2AF1206031206131205F912061A12C9
:10111A0005F91206211205F91217361206031206EC
:10112A00031205FEC2AF757C00757D0078FA79FA64
:10113A00308707D9FBD8F7021C00120F9A120FD377
:10114A001121112278988673120F1975A90075B6A4
:10115A0080757A0075881075890275C8247591049E
:10116A0075D84075A82275B80275E690759B80758A
:10117A009D0075D10E75BC5875BB0675BA1175E818
:10118A00801205EAD2AF1208A375360053DACF20CF
:10119A007E0343DA20307E0343DA1043DA01C2D8F1
:1011AA00C271120603D2617B037A0CE55B70077A7F
:1011BA000CDB0302112E1205F920700302112EC254
:1011CA0070E55CC3940240E1E52F541F855E5DF52E
:1011DA005EB55DD5DAD5C26153DACF207E0343DA34
:1011EA0020307E0343DA10C2D8C27178A2E67008B2
:1011FA00D274E52F54E0F52FC2757529001205FE49
:10120A00307409C3E529940A4002D2751205EF78B1
:10121A00023074027800C3E55C9840F0C2AF12064F
:10122A0013120613120613D2AF120603754C007876
:10123A0088E6B40302612E1205EF788CE6C39401A6
:10124A00500302132EE530C39401500302132E7586
:10125A007CA5757DF1207435C3E55C94FF500302CB
:10126A00132EC2AF120628D2AF1205FEC3E55C9454
:10127A000150EFC2AF1206131205F4120613D2AFD1
:10128A001205FEC3E55C94FF40E90217BB7F05D255
:10129A007F11221205FEC2AFC27F1122AE5CC3E5E6
:1012AA005C947FD2AF5002613E1205EAC2AF1206C9
:1012BA0028D2AFDFDA1159C3EE94057897F61206F1
:1012CA000312173E7F0AD27F11221205FEC2AFC255
:1012DA007F1122AE5CC3E55C947FD2AF50E6120563
:1012EA00EAC2AF1206131205F4120613D2AFDFD602
:1012FA001159EE24037896F6F87997E7C394824059
:10130A0003985006E824827897F612060312165BB1
:10131A0012176D1205FE1122C3E55C94FF500241BB
:10132A00590217BB757C00757D00C3E55C954C407E
:10133A0003855C4C1205FE78017988E7B4030278CC
:10134A0005C3E55C9840024139C2AF12062812066D
:10135A0028120628D2AF120603753000E4F531F5DB
:10136A00320531E531F4703F0532789AE67819147E
:10137A006012783214600D787D14600878FA14606F
:10138A0003753200C3E53298401D120F191205EA9F
:10139A00153275310078998673C2AF120628D2AF1A
:1013AA00789886731205FE1205F4E52A70053074E2
:1013BA0002212E78012074027806C3E55C9840A1C8
:1013CA007888E6C3940360031205FEE52A700302D7
:1013DA00112EC2AF120F19E4F522F523F524F525D3
:1013EA00F526F567D2AF7885E6C333F565E4F544AB
:1013FA00F545F546F547F548F570F52CF52DF53721
:10140A0075700875BB101205EA1208A730EDFDA821
:10141A00BDA9BEE97001F888711208AB757008752C
:10142A00BB10120F9AC2AF7561FF120921852261A2
:10143A00852262852263D2AF752201752401752542
:10144A0001752601856069756A0175B69075A903EB
:10145A00757A017888E6B40307C27D307602D27DB8
:0D146A00D268D269753300120E6E120E9F0B
:101477001209411209481209411209481209411279
:101487000BD6120709120CD7120D1E120948120BA0
:10149700C5306E0312070A20660312085D30660323
:1014A70012088D120CD7120D4D120948120BD630A7
:1014B7006E03120746120CD7120DC6120948120BFB
:1014C700C5306E031207A4120CD7120DF712094884
:1014D700120BD6306E03120801120CD7120E6E12C1
:1014E70009481208A7120BC5120CD7120E9F120833
:1014F700AB12094830692F8564618564628560692C
:10150700756A0179187A0CC3E53399400CC269D220
:101517006A8A357561FF02152DC3E55C94014003A6
:101527000214860215BB306A25206C22E53514703B
:1015370006C26AD26B8186F535C3E55C9401400328
:101547000214867888E6C3940360030215BB7536D8
:1015570000788279A4E760027803C3E55F98505466
:10156700307404E52A604D7888E6B40317207D05BA
:10157700207607A18B307602A18B206C07D26C8571
:10158700646181C578F0306C058564617820C3E5B6
:10159700419850028186306C1BC26CC27D30760246
:1015A700D27DD26A75351285646181860536E55C20
:1015B7006002A1BE753600C2AF120F197887E6FE2A
:1015C7007602120F9A7887EEF6E4F522F523F524D2
:1015D700F525F526F565752C00752D0075A900759F
:1015E700B680757A00D2AF1205FE120F1978A4E6FD
:1015F7006006C292C291C290307409C3E536940462
:101607004002212E6166901A0D782012169DE52062
:10161700B45A0CA312169DE520B4A50302163B7518
:101627007CA5757DF1120F2E12165B757C00757DFA
:101637000002165A901A0378807B0A12169DA30897
:10164700DBF9901A0F788C7B1912169DA308DBF92A
:10165700901A2822C2AF1216E01216BD901A007413
:101667000E1216A2A374091216A2A374151216A2BB
:10167700901A0378807B0A1216A1A308DBF9901A47
:101687000F788C7B191216A1A308DBF91216F31237
:1016970016D1901A2822E493F622E6438F01538F3E
:1016A700FDFFC3E583941C400122EF857CB7857D50
:1016B700B7F0538FFE22438F02438F01857CB78596
:1016C7007DB7901A0DF0538FFC22901A0D745AD1E2
:1016D700A2901A0E74A5D1A2227A3079D0782090E0
:1016E7001A40D19DE520F709A3DAF7227A3079D09D
:1016F700901A40E7D1A209A3DAF922AB74A875BB07
:1017070001027984BB02027985BB03027986BB0497
:10171700027992BB05027987BB060279A3BB070250
:10172700799CBB08027988BB09027989E8F7227C92
:1017370005120603DCFB22C2AF12061312061A12A9
:1017470006211206281205F412061312061A1206AB
:10175700211206281205F412061312061A12062180
:10176700120628D2AF22C2AF12062812062112068D
:101777001A1206131205F412062812062112061A67
:101787001206131205F412062812062112061A125F
:101797000613D2AF22AE74AF75C2AF12061312068C
:1017A700131206131205F4DEF21206281205F4DFEF
:1017B700F8D2AF22F13EF136F13675740175750135
:1017C700757600F19C7C05AD5C120603C3ED955C54
:1017D70070F5C3E55C9401400AC3E55C94FF4033B0
:1017E7000217F7F102D15BF13EC2AF75EF16F13682
:1017F700DCD50576C3E5769403500280C61217360A
:101807000575E5741490009F93F808C3E575985023
:101817000280AD1217361217360574C3E574940AA1
:1018270050028099120F2E12165BC2AF75EF161277
:02183700173662
:0319FD000210874E
:101A00000E0915FFFFFFFF03040A0301015AA50198
:101A1000FFFFFFFFFF03FFFFFF25D0FAFA04FF01DE
:091A2000007AFF0101000300FF40
:101A4000234F76736B794D5232304150726F2320A1
:101A500023424C48454C492346333930232020202B
:101A60002020202020202020202020202020202076
:101C0000C2AFC2D353D9BF7581C043B20343FF8073
:101C1000752438752503B1DC7529A5752AF175E29F
:101C20004043F18053A47F75D4FFD2877DFA7803B7
:101C300079E67C10752200752300901DE97B0675FE
:101C400024987525013087028145208708D8FBD963
:101C5000F9DCF781B7308708D8FBD9F9DCF781B711
:101C6000B19CE493A3C39A6004DDC381B7DBDBB10D
:101C70008E6002812E7B08E493FAA3B16FDBF87AC1
:101C800030B16F752200752300B18EEAFCEBFDC305
:101C9000ED94FE400EB18E8A278B28ED30E0048A49
:101CA000828B83B18E7AC270D8C3ED94FE601950D6
:101CB000CEBD002BEC600F7520007521FF7529004B
:101CC000752A000200008100A827A9280809D80465
:101CD000D90281DCB192EA89AAF281CE0D81A3C337
:101CE000ED94035053EDA2E092007AC5C3E58294CF
:101CF00000E583941C508A200010438F02438F011B
:101D00008529B7852AB7F0300029A827A92808090E
:101D1000438F01538FFDD804D902A133C3E58394C7
:101D20001C4003A3A11689AAE28529B7852AB7F02A
:101D3000A3A116538FFC817F7AC1BD030CE493A34A
:101D4000FAB153DCF8B14B817F8181AA22AB23B178
:101D50006FEBFAEA6222752608C3E52313F523E543
:101D60002213F52250066323A0632201D526EAB18F
:101D7000DCB1DC75260AEAF4200102D287300102C8
:101D8000C287B1DCC3134002C201D526EB22B19257
:101D9000EAFB208702A192308702A197752608AE40
:101DA00024AF25C3EF13FFEE13FEB1E0B1DCC3EAAD
:101DB000133087024480FA30E703632201C3E5232E
:101DC00013F523E52213F52250066323A0632201B5
:101DD000D526D9E52265236523F52222AE24AF2539
:101DE0000E0FDEFEDFFCD20122424C48656C6934E6
:071DF000373164F390060196
:00000001FF
